 management_agent

 Timestamp is ffffffff (Sun Feb  7 06:28:15 2106)

 Preferred load address is 10000000

 Start         Length     Name                   Class
 0001:00000000 00000ffaH .text$mn                CODE
 0002:00000000 000000c0H .idata$5                DATA
 0002:000000c0 00000004H .00cfg                  DATA
 0002:000000c4 00000004H .CRT$XCA                DATA
 0002:000000c8 00000004H .CRT$XCZ                DATA
 0002:000000cc 00000004H .CRT$XIA                DATA
 0002:000000d0 00000004H .CRT$XIZ                DATA
 0002:000000d4 00000004H .CRT$XPA                DATA
 0002:000000d8 00000004H .CRT$XPZ                DATA
 0002:000000dc 00000004H .CRT$XTA                DATA
 0002:000000e0 00000010H .CRT$XTZ                DATA
 0002:000000e4 00000000H .gfids$y                DATA
 0002:000000f0 00000220H .rdata                  DATA
 0002:00000310 00000004H .rdata$sxdata           DATA
 0002:00000314 00000290H .rdata$zzzdbg           DATA
 0002:000005a4 00000004H .rtc$IAA                DATA
 0002:000005a8 00000004H .rtc$IZZ                DATA
 0002:000005ac 00000004H .rtc$TAA                DATA
 0002:000005b0 00000008H .rtc$TZZ                DATA
 0002:000005b8 00000088H .xdata$x                DATA
 0002:00000640 00000120H .edata                  DATA
 0002:00000760 0000008cH .idata$2                DATA
 0002:000007ec 00000014H .idata$3                DATA
 0002:00000800 000000c0H .idata$4                DATA
 0002:000008c0 00000436H .idata$6                DATA
 0003:00000000 00000018H .data                   DATA
 0003:00000018 00000374H .bss                    DATA
 0004:00000000 00000060H .rsrc$01                DATA
 0004:00000060 00000338H .rsrc$02                DATA

  Address         Publics by Value              Rva+Base       Lib:Object

 0000:00000000       ___guard_iat_count         00000000     <absolute>
 0000:00000000       ___hybrid_auxiliary_iat    00000000     <absolute>
 0000:00000000       ___hybrid_code_map         00000000     <absolute>
 0000:00000000       ___guard_iat_table         00000000     <absolute>
 0000:00000000       ___hybrid_code_map_count   00000000     <absolute>
 0000:00000000       ___guard_longjmp_table     00000000     <absolute>
 0000:00000000       ___volatile_metadata       00000000     <absolute>
 0000:00000000       ___enclave_config          00000000     <absolute>
 0000:00000000       ___guard_fids_count        00000000     <absolute>
 0000:00000000       ___guard_fids_table        00000000     <absolute>
 0000:00000000       ___guard_longjmp_count     00000000     <absolute>
 0000:00000000       ___dynamic_value_reloc_table 00000000     <absolute>
 0000:00000001       ___safe_se_handler_count   00000001     <absolute>
 0000:00000100       ___guard_flags             00000100     <absolute>
 0000:00000000       ___ImageBase               10000000     <linker-defined>
 0001:00000000       _JNI_OnLoad@8              10001000 f   FileSystemImpl.obj
 0001:00000027       _Java_jdk_internal_agent_FileSystemImpl_init0@8 10001027 f   FileSystemImpl.obj
 0001:0000002a       _Java_jdk_internal_agent_FileSystemImpl_isAccessUserOnly0@12 1000102a f   FileSystemImpl.obj
 0001:000000c4       _Java_jdk_internal_agent_FileSystemImpl_isSecuritySupported0@12 100010c4 f   FileSystemImpl.obj
 0001:00000370       _JNU_ThrowOutOfMemoryError@8 10001370 f   java:java.dll
 0001:00000376       _JNU_ThrowInternalError@8  10001376 f   java:java.dll
 0001:0000037c       _JNU_ThrowIOException@8    1000137c f   java:java.dll
 0001:00000382       _JNU_ThrowIOExceptionWithLastError@8 10001382 f   java:java.dll
 0001:00000388       _JNU_GetStringPlatformChars@12 10001388 f   java:java.dll
 0001:0000038e       _JNU_ReleaseStringPlatformChars@12 1000138e f   java:java.dll
 0001:00000394       @__security_check_cookie@4 10001394 f   MSVCRT:secchk.obj
 0001:000006c5       __DllMainCRTStartup@12     100016c5 f   MSVCRT:dll_dllmain.obj
 0001:000006e8       ___raise_securityfailure   100016e8 f   MSVCRT:gs_report.obj
 0001:00000710       ___report_gsfailure        10001710 f   MSVCRT:gs_report.obj
 0001:00000856       ___security_init_cookie    10001856 f   MSVCRT:gs_support.obj
 0001:000008a1       _DllMain@12                100018a1 f   MSVCRT:dll_dllmain_stub.obj
 0001:000008c3       ?__scrt_initialize_type_info@@YAXXZ 100018c3 f   MSVCRT:tncleanup.obj
 0001:000008cf       ?__scrt_uninitialize_type_info@@YAXXZ 100018cf f   MSVCRT:tncleanup.obj
 0001:000008db       ___local_stdio_printf_options 100018db f i MSVCRT:default_local_stdio_options.obj
 0001:000008e1       ___local_stdio_scanf_options 100018e1 f i MSVCRT:default_local_stdio_options.obj
 0001:000008e7       ___scrt_initialize_default_local_stdio_options 100018e7 f   MSVCRT:default_local_stdio_options.obj
 0001:00000948       ___scrt_acquire_startup_lock 10001948 f   MSVCRT:utility.obj
 0001:0000097a       ___scrt_dllmain_after_initialize_c 1000197a f   MSVCRT:utility.obj
 0001:000009a5       ___scrt_dllmain_before_initialize_c 100019a5 f   MSVCRT:utility.obj
 0001:000009b3       ___scrt_dllmain_crt_thread_attach 100019b3 f   MSVCRT:utility.obj
 0001:000009d2       ___scrt_dllmain_crt_thread_detach 100019d2 f   MSVCRT:utility.obj
 0001:000009df       ___scrt_dllmain_exception_filter 100019df f   MSVCRT:utility.obj
 0001:00000a13       ___scrt_dllmain_uninitialize_c 10001a13 f   MSVCRT:utility.obj
 0001:00000a36       ___scrt_dllmain_uninitialize_critical 10001a36 f   MSVCRT:utility.obj
 0001:00000a43       ___scrt_initialize_crt     10001a43 f   MSVCRT:utility.obj
 0001:00000a7c       ___scrt_initialize_onexit_tables 10001a7c f   MSVCRT:utility.obj
 0001:00000b21       ___scrt_is_nonwritable_in_current_image 10001b21 f   MSVCRT:utility.obj
 0001:00000bb5       ___scrt_release_startup_lock 10001bb5 f   MSVCRT:utility.obj
 0001:00000bd2       ___scrt_uninitialize_crt   10001bd2 f   MSVCRT:utility.obj
 0001:00000bfa       ___scrt_get_dyn_tls_init_callback 10001bfa f   MSVCRT:dyn_tls_init.obj
 0001:00000c00       ___scrt_fastfail           10001c00 f   MSVCRT:utility_desktop.obj
 0001:00000d1a       __crt_debugger_hook        10001d1a f   MSVCRT:utility_desktop.obj
 0001:00000d22       __RTC_Initialize           10001d22 f   MSVCRT:initsect.obj
 0001:00000d4e       __RTC_Terminate            10001d4e f   MSVCRT:initsect.obj
 0001:00000d80       __SEH_prolog4              10001d80 f   MSVCRT:sehprolg4.obj
 0001:00000dc6       __SEH_epilog4              10001dc6 f   MSVCRT:sehprolg4.obj
 0001:00000ddb       __except_handler4          10001ddb f   MSVCRT:chandler4gs.obj
 0001:00000dfe       @_guard_check_icall_nop@4  10001dfe f i MSVCRT:guard_support.obj
 0001:00000dff       ___isa_available_init      10001dff f   MSVCRT:cpu_disp.obj
 0001:00000f96       __get_startup_argv_mode    10001f96 f   MSVCRT:argv_mode.obj
 0001:00000f9a       ___scrt_is_ucrt_dll_in_use 10001f9a f   MSVCRT:ucrt_detection.obj
 0001:00000fa6       _IsProcessorFeaturePresent@4 10001fa6 f   kernel32:KERNEL32.dll
 0001:00000fac       _strchr                    10001fac f   vcruntime:VCRUNTIME140.dll
 0001:00000fb2       ___std_type_info_destroy_list 10001fb2 f   vcruntime:VCRUNTIME140.dll
 0001:00000fb8       _memset                    10001fb8 f   vcruntime:VCRUNTIME140.dll
 0001:00000fbe       __except_handler4_common   10001fbe f   vcruntime:VCRUNTIME140.dll
 0001:00000fc4       __initterm                 10001fc4 f   ucrt:api-ms-win-crt-runtime-l1-1-0.dll
 0001:00000fca       __initterm_e               10001fca f   ucrt:api-ms-win-crt-runtime-l1-1-0.dll
 0001:00000fd0       __seh_filter_dll           10001fd0 f   ucrt:api-ms-win-crt-runtime-l1-1-0.dll
 0001:00000fd6       __configure_narrow_argv    10001fd6 f   ucrt:api-ms-win-crt-runtime-l1-1-0.dll
 0001:00000fdc       __initialize_narrow_environment 10001fdc f   ucrt:api-ms-win-crt-runtime-l1-1-0.dll
 0001:00000fe2       __initialize_onexit_table  10001fe2 f   ucrt:api-ms-win-crt-runtime-l1-1-0.dll
 0001:00000fe8       __execute_onexit_table     10001fe8 f   ucrt:api-ms-win-crt-runtime-l1-1-0.dll
 0001:00000fee       __cexit                    10001fee f   ucrt:api-ms-win-crt-runtime-l1-1-0.dll
 0001:00000ff4       ___scrt_stub_for_acrt_uninitialize_critical 10001ff4 f   MSVCRT:ucrt_stubs.obj
 0001:00000ff4       ___acrt_thread_detach      10001ff4 f   MSVCRT:ucrt_stubs.obj
 0001:00000ff4       ___scrt_stub_for_acrt_thread_detach 10001ff4 f   MSVCRT:ucrt_stubs.obj
 0001:00000ff4       ___acrt_uninitialize       10001ff4 f   MSVCRT:ucrt_stubs.obj
 0001:00000ff4       ___scrt_stub_for_acrt_uninitialize 10001ff4 f   MSVCRT:ucrt_stubs.obj
 0001:00000ff4       ___scrt_stub_for_acrt_initialize 10001ff4 f   MSVCRT:ucrt_stubs.obj
 0001:00000ff4       ___vcrt_thread_detach      10001ff4 f   MSVCRT:ucrt_stubs.obj
 0001:00000ff4       ___acrt_uninitialize_critical 10001ff4 f   MSVCRT:ucrt_stubs.obj
 0001:00000ff4       ___vcrt_thread_attach      10001ff4 f   MSVCRT:ucrt_stubs.obj
 0001:00000ff4       ___scrt_stub_for_acrt_thread_attach 10001ff4 f   MSVCRT:ucrt_stubs.obj
 0001:00000ff4       ___vcrt_uninitialize       10001ff4 f   MSVCRT:ucrt_stubs.obj
 0001:00000ff4       ___vcrt_uninitialize_critical 10001ff4 f   MSVCRT:ucrt_stubs.obj
 0001:00000ff4       ___vcrt_initialize         10001ff4 f   MSVCRT:ucrt_stubs.obj
 0001:00000ff4       ___acrt_initialize         10001ff4 f   MSVCRT:ucrt_stubs.obj
 0001:00000ff4       ___acrt_thread_attach      10001ff4 f   MSVCRT:ucrt_stubs.obj
 0001:00000ff7       __is_c_termination_complete 10001ff7 f   MSVCRT:ucrt_stubs.obj
 0001:00000ff7       ___scrt_stub_for_is_c_termination_complete 10001ff7 f   MSVCRT:ucrt_stubs.obj
 0002:00000000       __imp__GetFileSecurityA@20 10002000     advapi32:ADVAPI32.dll
 0002:00000004       __imp__GetSecurityDescriptorOwner@12 10002004     advapi32:ADVAPI32.dll
 0002:00000008       __imp__GetSecurityDescriptorDacl@16 10002008     advapi32:ADVAPI32.dll
 0002:0000000c       __imp__GetAclInformation@16 1000200c     advapi32:ADVAPI32.dll
 0002:00000010       __imp__GetAce@12           10002010     advapi32:ADVAPI32.dll
 0002:00000014       __imp__EqualSid@8          10002014     advapi32:ADVAPI32.dll
 0002:00000018       \177ADVAPI32_NULL_THUNK_DATA 10002018     advapi32:ADVAPI32.dll
 0002:0000001c       __imp__GetSystemTimeAsFileTime@4 1000201c     kernel32:KERNEL32.dll
 0002:00000020       __imp__DisableThreadLibraryCalls@4 10002020     kernel32:KERNEL32.dll
 0002:00000024       __imp__InitializeSListHead@4 10002024     kernel32:KERNEL32.dll
 0002:00000028       __imp__IsDebuggerPresent@0 10002028     kernel32:KERNEL32.dll
 0002:0000002c       __imp__GetCurrentThreadId@0 1000202c     kernel32:KERNEL32.dll
 0002:00000030       __imp__GetVolumeInformationA@32 10002030     kernel32:KERNEL32.dll
 0002:00000034       __imp__GetLastError@0      10002034     kernel32:KERNEL32.dll
 0002:00000038       __imp__UnhandledExceptionFilter@4 10002038     kernel32:KERNEL32.dll
 0002:0000003c       __imp__SetUnhandledExceptionFilter@4 1000203c     kernel32:KERNEL32.dll
 0002:00000040       __imp__GetCurrentProcess@0 10002040     kernel32:KERNEL32.dll
 0002:00000044       __imp__TerminateProcess@8  10002044     kernel32:KERNEL32.dll
 0002:00000048       __imp__IsProcessorFeaturePresent@4 10002048     kernel32:KERNEL32.dll
 0002:0000004c       __imp__QueryPerformanceCounter@4 1000204c     kernel32:KERNEL32.dll
 0002:00000050       __imp__GetCurrentProcessId@0 10002050     kernel32:KERNEL32.dll
 0002:00000054       \177KERNEL32_NULL_THUNK_DATA 10002054     kernel32:KERNEL32.dll
 0002:00000058       __imp__memset              10002058     vcruntime:VCRUNTIME140.dll
 0002:0000005c       __imp____std_type_info_destroy_list 1000205c     vcruntime:VCRUNTIME140.dll
 0002:00000060       __imp__strchr              10002060     vcruntime:VCRUNTIME140.dll
 0002:00000064       __imp___except_handler4_common 10002064     vcruntime:VCRUNTIME140.dll
 0002:00000068       \177VCRUNTIME140_NULL_THUNK_DATA 10002068     vcruntime:VCRUNTIME140.dll
 0002:0000006c       __imp__free                1000206c     ucrt:api-ms-win-crt-heap-l1-1-0.dll
 0002:00000070       __imp__malloc              10002070     ucrt:api-ms-win-crt-heap-l1-1-0.dll
 0002:00000074       \177api-ms-win-crt-heap-l1-1-0_NULL_THUNK_DATA 10002074     ucrt:api-ms-win-crt-heap-l1-1-0.dll
 0002:00000078       __imp___cexit              10002078     ucrt:api-ms-win-crt-runtime-l1-1-0.dll
 0002:0000007c       __imp___execute_onexit_table 1000207c     ucrt:api-ms-win-crt-runtime-l1-1-0.dll
 0002:00000080       __imp___initialize_onexit_table 10002080     ucrt:api-ms-win-crt-runtime-l1-1-0.dll
 0002:00000084       __imp___initterm           10002084     ucrt:api-ms-win-crt-runtime-l1-1-0.dll
 0002:00000088       __imp___initterm_e         10002088     ucrt:api-ms-win-crt-runtime-l1-1-0.dll
 0002:0000008c       __imp___seh_filter_dll     1000208c     ucrt:api-ms-win-crt-runtime-l1-1-0.dll
 0002:00000090       __imp___configure_narrow_argv 10002090     ucrt:api-ms-win-crt-runtime-l1-1-0.dll
 0002:00000094       __imp___initialize_narrow_environment 10002094     ucrt:api-ms-win-crt-runtime-l1-1-0.dll
 0002:00000098       \177api-ms-win-crt-runtime-l1-1-0_NULL_THUNK_DATA 10002098     ucrt:api-ms-win-crt-runtime-l1-1-0.dll
 0002:0000009c       __imp__strdup              1000209c     ucrt:api-ms-win-crt-string-l1-1-0.dll
 0002:0000009c       __imp___strdup             1000209c     ucrt:api-ms-win-crt-string-l1-1-0.dll
 0002:000000a0       \177api-ms-win-crt-string-l1-1-0_NULL_THUNK_DATA 100020a0     ucrt:api-ms-win-crt-string-l1-1-0.dll
 0002:000000a4       __imp__JNU_ReleaseStringPlatformChars@12 100020a4     java:java.dll
 0002:000000a8       __imp__JNU_GetStringPlatformChars@12 100020a8     java:java.dll
 0002:000000ac       __imp__JNU_ThrowIOExceptionWithLastError@8 100020ac     java:java.dll
 0002:000000b0       __imp__JNU_ThrowIOException@8 100020b0     java:java.dll
 0002:000000b4       __imp__JNU_ThrowInternalError@8 100020b4     java:java.dll
 0002:000000b8       __imp__JNU_ThrowOutOfMemoryError@8 100020b8     java:java.dll
 0002:000000bc       \177java_NULL_THUNK_DATA   100020bc     java:java.dll
 0002:000000c0       ___guard_check_icall_fptr  100020c0     MSVCRT:guard_support.obj
 0002:000000c4       ___xc_a                    100020c4     MSVCRT:initializers.obj
 0002:000000c8       ___xc_z                    100020c8     MSVCRT:initializers.obj
 0002:000000cc       ___xi_a                    100020cc     MSVCRT:initializers.obj
 0002:000000d0       ___xi_z                    100020d0     MSVCRT:initializers.obj
 0002:000000d4       ___xp_a                    100020d4     MSVCRT:initializers.obj
 0002:000000d8       ___xp_z                    100020d8     MSVCRT:initializers.obj
 0002:000000dc       ___xt_a                    100020dc     MSVCRT:initializers.obj
 0002:000000e0       ___xt_z                    100020e0     MSVCRT:initializers.obj
 0002:000000f0       ??_C@_0O@PNKFDMOJ@Malformed?5UNC@ 100020f0     FileSystemImpl.obj
 0002:00000100       ??_C@_0CA@CGFDCJE@Absolute?5filename?5not?5specified@ 10002100     FileSystemImpl.obj
 0002:00000120       ??_C@_0BM@JPGKFFDK@GetVolumeInformation?5failed@ 10002120     FileSystemImpl.obj
 0002:0000013c       ??_C@_0BH@EKMPGKNN@GetFileSecurity?5failed@ 1000213c     FileSystemImpl.obj
 0002:00000154       ??_C@_0CC@PLIGLKOL@GetSecurityDescriptorOwner?5fail@ 10002154     FileSystemImpl.obj
 0002:00000178       ??_C@_0CB@EKBMIJAO@GetSecurityDescriptorDacl?5faile@ 10002178     FileSystemImpl.obj
 0002:0000019c       ??_C@_0CM@JFCPAEMB@Security?5descriptor?5does?5not?5co@ 1000219c     FileSystemImpl.obj
 0002:000001c8       ??_C@_0BJ@OEDGCHLN@GetAclInformation?5failed@ 100021c8     FileSystemImpl.obj
 0002:000001e4       ??_C@_0O@HNKFIIOB@GetAce?5failed@ 100021e4     FileSystemImpl.obj
 0002:000001f4       __pDefaultRawDllMain       100021f4     MSVCRT:dll_dllmain.obj
 0002:000001f4       __pRawDllMain              100021f4     MSVCRT:dll_dllmain.obj
 0002:00000270       __load_config_used         10002270     MSVCRT:loadcfg.obj
 0002:00000310       ___safe_se_handler_table   10002310     <linker-defined>
 0002:000005a4       ___rtc_iaa                 100025a4     MSVCRT:initsect.obj
 0002:000005a8       ___rtc_izz                 100025a8     MSVCRT:initsect.obj
 0002:000005ac       ___rtc_taa                 100025ac     MSVCRT:initsect.obj
 0002:000005b0       ___rtc_tzz                 100025b0     MSVCRT:initsect.obj
 0002:00000760       __IMPORT_DESCRIPTOR_java   10002760     java:java.dll
 0002:00000774       __IMPORT_DESCRIPTOR_ADVAPI32 10002774     advapi32:ADVAPI32.dll
 0002:00000788       __IMPORT_DESCRIPTOR_KERNEL32 10002788     kernel32:KERNEL32.dll
 0002:0000079c       __IMPORT_DESCRIPTOR_VCRUNTIME140 1000279c     vcruntime:VCRUNTIME140.dll
 0002:000007b0       __IMPORT_DESCRIPTOR_api-ms-win-crt-heap-l1-1-0 100027b0     ucrt:api-ms-win-crt-heap-l1-1-0.dll
 0002:000007c4       __IMPORT_DESCRIPTOR_api-ms-win-crt-runtime-l1-1-0 100027c4     ucrt:api-ms-win-crt-runtime-l1-1-0.dll
 0002:000007d8       __IMPORT_DESCRIPTOR_api-ms-win-crt-string-l1-1-0 100027d8     ucrt:api-ms-win-crt-string-l1-1-0.dll
 0002:000007ec       __NULL_IMPORT_DESCRIPTOR   100027ec     java:java.dll
 0003:00000000       ___security_cookie_complement 10003000     MSVCRT:gs_cookie.obj
 0003:00000004       ___security_cookie         10003004     MSVCRT:gs_cookie.obj
 0003:00000008       ___scrt_native_dllmain_reason 10003008     MSVCRT:utility.obj
 0003:00000010       ___isa_enabled             10003010     MSVCRT:cpu_disp.obj
 0003:00000014       ___scrt_ucrt_dll_is_in_use 10003014     MSVCRT:ucrt_stubs.obj
 0003:00000340       ?__type_info_root_node@@3U__type_info_node@@A 10003340     MSVCRT:tncleanup.obj
 0003:00000348       ?_OptionsStorage@?1??__local_stdio_printf_options@@9@4_KA 10003348     MSVCRT:default_local_stdio_options.obj
 0003:00000350       ?_OptionsStorage@?1??__local_stdio_scanf_options@@9@4_KA 10003350     MSVCRT:default_local_stdio_options.obj
 0003:00000358       ___scrt_current_native_startup_state 10003358     MSVCRT:utility.obj
 0003:0000035c       ___scrt_native_startup_lock 1000335c     MSVCRT:utility.obj
 0003:0000037c       ___scrt_debugger_hook_flag 1000337c     MSVCRT:utility_desktop.obj
 0003:00000380       ___isa_available           10003380     MSVCRT:cpu_disp.obj
 0003:00000384       ___favor                   10003384     MSVCRT:cpu_disp.obj
 0003:00000388       ___dyn_tls_init_callback   10003388     <common>

 entry point at        0001:000006c5

 Static symbols

 0000:ffffa000       .debug$S                   10000000     kernel32:KERNEL32.dll
 0000:ffffa000       .debug$S                   10000000     kernel32:KERNEL32.dll
 0000:ffffa000       .debug$S                   10000000     kernel32:KERNEL32.dll
 0000:ffffa000       .debug$S                   10000000     kernel32:KERNEL32.dll
 0000:ffffa000       .debug$S                   10000000     java:java.dll
 0000:ffffa000       .debug$S                   10000000     java:java.dll
 0000:ffffa000       .debug$S                   10000000     java:java.dll
 0000:ffffa000       .debug$S                   10000000     java:java.dll
 0000:ffffa000       .debug$S                   10000000     java:java.dll
 0000:ffffa000       .debug$S                   10000000     management_agent.exp
 0000:ffffa000       .debug$S                   10000000     java:java.dll
 0000:ffffa000       .debug$S                   10000000     advapi32:ADVAPI32.dll
 0000:ffffa000       .debug$S                   10000000     advapi32:ADVAPI32.dll
 0000:ffffa000       .debug$S                   10000000     advapi32:ADVAPI32.dll
 0000:ffffa000       .debug$S                   10000000     ucrt:api-ms-win-crt-string-l1-1-0.dll
 0000:ffffa000       .debug$S                   10000000     ucrt:api-ms-win-crt-runtime-l1-1-0.dll
 0000:ffffa000       .debug$S                   10000000     ucrt:api-ms-win-crt-runtime-l1-1-0.dll
 0000:ffffa000       .debug$S                   10000000     ucrt:api-ms-win-crt-runtime-l1-1-0.dll
 0000:ffffa000       .debug$S                   10000000     ucrt:api-ms-win-crt-runtime-l1-1-0.dll
 0000:ffffa000       .debug$S                   10000000     ucrt:api-ms-win-crt-runtime-l1-1-0.dll
 0000:ffffa000       .debug$S                   10000000     ucrt:api-ms-win-crt-runtime-l1-1-0.dll
 0000:ffffa000       .debug$S                   10000000     ucrt:api-ms-win-crt-runtime-l1-1-0.dll
 0000:ffffa000       .debug$S                   10000000     ucrt:api-ms-win-crt-runtime-l1-1-0.dll
 0000:ffffa000       .debug$S                   10000000     ucrt:api-ms-win-crt-runtime-l1-1-0.dll
 0000:ffffa000       .debug$S                   10000000     ucrt:api-ms-win-crt-runtime-l1-1-0.dll
 0000:ffffa000       .debug$S                   10000000     ucrt:api-ms-win-crt-runtime-l1-1-0.dll
 0000:ffffa000       .debug$S                   10000000     ucrt:api-ms-win-crt-runtime-l1-1-0.dll
 0000:ffffa000       .debug$S                   10000000     ucrt:api-ms-win-crt-heap-l1-1-0.dll
 0000:ffffa000       .debug$S                   10000000     ucrt:api-ms-win-crt-heap-l1-1-0.dll
 0000:ffffa000       .debug$S                   10000000     advapi32:ADVAPI32.dll
 0000:ffffa000       .debug$S                   10000000     vcruntime:VCRUNTIME140.dll
 0000:ffffa000       .debug$S                   10000000     vcruntime:VCRUNTIME140.dll
 0000:ffffa000       .debug$S                   10000000     vcruntime:VCRUNTIME140.dll
 0000:ffffa000       .debug$S                   10000000     vcruntime:VCRUNTIME140.dll
 0000:ffffa000       .debug$S                   10000000     advapi32:ADVAPI32.dll
 0000:ffffa000       .debug$S                   10000000     kernel32:KERNEL32.dll
 0000:ffffa000       .debug$S                   10000000     kernel32:KERNEL32.dll
 0000:ffffa000       .debug$S                   10000000     kernel32:KERNEL32.dll
 0000:ffffa000       .debug$S                   10000000     kernel32:KERNEL32.dll
 0000:ffffa000       .debug$S                   10000000     kernel32:KERNEL32.dll
 0000:ffffa000       .debug$S                   10000000     kernel32:KERNEL32.dll
 0000:ffffa000       .debug$S                   10000000     kernel32:KERNEL32.dll
 0000:ffffa000       .debug$S                   10000000     kernel32:KERNEL32.dll
 0000:ffffa000       .debug$S                   10000000     kernel32:KERNEL32.dll
 0000:ffffa000       .debug$S                   10000000     kernel32:KERNEL32.dll
 0000:ffffa000       .debug$S                   10000000     kernel32:KERNEL32.dll
 0000:ffffa000       .debug$S                   10000000     kernel32:KERNEL32.dll
 0000:ffffa000       .debug$S                   10000000     advapi32:ADVAPI32.dll
 0001:0000010a       _getFileDACL               1000110a f   FileSystemImpl.obj
 0001:00000154       _getFileSecurityDescriptor 10001154 f   FileSystemImpl.obj
 0001:000001db       _isAccessUserOnly          100011db f   FileSystemImpl.obj
 0001:0000028d       _isSecuritySupported       1000128d f   FileSystemImpl.obj
 0001:000003a5       ?dllmain_crt_dispatch@@YGHQAUHINSTANCE__@@KQAX@Z 100013a5 f   MSVCRT:dll_dllmain.obj
 0001:000003f8       ?dllmain_crt_process_attach@@YAHQAUHINSTANCE__@@QAX@Z 100013f8 f   MSVCRT:dll_dllmain.obj
 0001:00000502       ?dllmain_crt_process_detach@@YAH_N@Z 10001502 f   MSVCRT:dll_dllmain.obj
 0001:00000594       ?dllmain_dispatch@@YAHQAUHINSTANCE__@@KQAX@Z 10001594 f   MSVCRT:dll_dllmain.obj
 0001:0000069a       ?dllmain_raw@@YGHQAUHINSTANCE__@@KQAX@Z 1000169a f   MSVCRT:dll_dllmain.obj
 0001:00000809       ___get_entropy             10001809 f   MSVCRT:gs_support.obj
 0001:00000904       ?find_pe_section@@YAPAU_IMAGE_SECTION_HEADER@@QAEI@Z 10001904 f   MSVCRT:utility.obj
 0001:00000d80       $$000000                   10001d80     MSVCRT:sehprolg4.obj
 0002:000001f8       _GS_ExceptionPointers      100021f8     MSVCRT:gs_report.obj
 0002:000005b8       __sehtable$?dllmain_crt_process_attach@@YAHQAUHINSTANCE__@@QAX@Z 100025b8     MSVCRT:dll_dllmain.obj
 0002:000005d8       __sehtable$?dllmain_crt_process_detach@@YAH_N@Z 100025d8     MSVCRT:dll_dllmain.obj
 0002:000005f8       __sehtable$?dllmain_dispatch@@YAHQAUHINSTANCE__@@KQAX@Z 100025f8     MSVCRT:dll_dllmain.obj
 0002:00000618       __sehtable$___scrt_is_nonwritable_in_current_image 10002618     MSVCRT:utility.obj
 0002:00000640       .edata                     10002640     management_agent.exp
 0002:00000668       rgpv                       10002668     management_agent.exp
 0002:00000678       rgszName                   10002678     management_agent.exp
 0002:00000688       rgwOrd                     10002688     management_agent.exp
 0002:00000690       szName                     10002690     management_agent.exp
 0002:000006a5       $N00001                    100026a5     management_agent.exp
 0002:000006b3       $N00002                    100026b3     management_agent.exp
 0002:000006e3       $N00003                    100026e3     management_agent.exp
 0002:00000720       $N00004                    10002720     management_agent.exp
 0002:00000986       .idata$6                   10002986     java:java.dll
 0002:00000a08       .idata$6                   10002a08     advapi32:ADVAPI32.dll
 0002:00000b62       .idata$6                   10002b62     kernel32:KERNEL32.dll
 0002:00000bbe       .idata$6                   10002bbe     vcruntime:VCRUNTIME140.dll
 0002:00000c92       .idata$6                   10002c92     ucrt:api-ms-win-crt-heap-l1-1-0.dll
 0002:00000cb2       .idata$6                   10002cb2     ucrt:api-ms-win-crt-runtime-l1-1-0.dll
 0002:00000cd4       .idata$6                   10002cd4     ucrt:api-ms-win-crt-string-l1-1-0.dll
 0003:00000018       ?__proc_attached@@3HA      10003018     MSVCRT:dll_dllmain.obj
 0003:00000020       _GS_ExceptionRecord        10003020     MSVCRT:gs_report.obj
 0003:00000070       _GS_ContextRecord          10003070     MSVCRT:gs_report.obj
 0003:00000360       ?is_initialized_as_dll@@3_NA 10003360     MSVCRT:utility.obj
 0003:00000361       ?module_local_atexit_table_initialized@@3_NA 10003361     MSVCRT:utility.obj
 0003:00000364       ?module_local_atexit_table@@3U_onexit_table_t@@A 10003364     MSVCRT:utility.obj
 0003:00000370       ?module_local_at_quick_exit_table@@3U_onexit_table_t@@A 10003370     MSVCRT:utility.obj
 0004:00000060       $R000000                   10004060     management_agent.dll.res
